:15010000AD401718300EAD401710FB200E01A9FF20A01E386034
:200200004C85024CBD024C5A1E4CA01E4C00015F1800800486C3900586C391C260B1C2A0FD
:20022000006062036403D80305043304FD039F0542093F097A05FC0695059F059F05BD0818
:20024000C1088A089B08E90861055105410852084F086208E707CD0406059F051506A7055A
:20026000B704BF048306A1049F059F05A8064F094D090707AA023705BD021B09B10820413B
:200280005420807009A90085208522A90B85218523A001B122AA49FF9122D122088A9122A9
:2002A000E622D002E62328F0EA88D8A5206D130285249865218525989120C89120A5228533
:2002C000C68526A52385C78527208706AD8302852AAD8402852BA98085C1A93085C0A2004D
:2002E00086BE86C2CA9AD820F90420F2024CE6028365C930B07BC908900C0AAABD1F02487E
:20030000BD1E0248084065C1AAB1C148B50091C168950060208706A921200902A52A38EDEC
:200320008302AAA52BED840220A005A5BEF012A97E852AA902852B20A104A628A52920A0CF
:2003400005A907200902208706A52685C6A52785C74CCC02A27CE4C190BAA6C1E6C1E6C106
:200360001860C6BDA5BDF0ACA5BC852AA5BD852B60C940B0434820F9046D830285BC6848BE
:2003800029076D840285BD682908D0DCA5BCA62A852A86BCA5BDA62B852B86BDA5C6E90116
:2003A00085C6B002C6C7C524A5C7E52590AAA5BC91C6C8A5BD91C660484A4A4A4A290EAA30
:2003C00068C960291FB00209E018F007652A85BC98652B85BD4CFC02A52C85B8A52D85B9F8
:2003E000202504201404512AAA20F9048AF0F10AF012A5B8852CA5B9852D4C6403202504A9
:20040000C90DD0F660202504C95BB0EEC94190EA0A208705A000B12CE62CD002E62DC90D51
:200420001860201404B12CC920F0F7C93A181002C9306020250490C284BC84BDA5BCA6BDF9
:2004400006BC26BD06BC26BD1865BC85BC8A65BD06BC2A85BD201404290F65BC85BC98652F
:20046000BD85BD202504B0D44C800520FC06A5BC05BDF048A520852CA521852D206D05F0F2
:2004800012A528C5BCA529E5BDB008201404D0FB4C7C04A52845BCD004A52945BD6020A66D
:2004A0000420F90410F8E6BF30034C0902C6BF60C922F0FB20A604201404D0F44C1403A957
:2004C0002020A604A5BF298730E5D0F360A27B205603E6C1E6C1E6C138B503F5009500B52C
:2004E00004F501500449800901300AD0041500F002560256025602900CA000B12AE62AD0C7
:2005000002E62B090060A5BEF028201404D0FB206D05F01B204C05200C02B009A5C4852AD4
:20052000A5C5852B60AD8302852AAD8402852B4C140385BF4C4903A520852CA521852D2030
:200540006D05F0EBA52A85C4A52B85C5A90185BE60206B04F0BEA5BC8528A5BD85294C1414
:200560000320FD0820F408207404D0EA602014048528201404852905286020FC0620800566
:20058000A5BD208705A5BCA6C1CA950086C1E4C0D00D4C1403A6C1E08010F7B500E6C16071
:2005A00085BD86BC4CB805A6C1B5011008204108A92D20A60420FC06A91F85B885BAA92A37
:2005C00085B985BBA6BCA4BD38E6B88AE910AA98E927A8B0F4C6B98A69E8AA986903A890A3
:2005E000F48A38E6BAE964B0FA8810F6C6BB690A90FA093085BCA92085BDA2FB86C3B5BDC5
:2006000005BDC920F009A03084BD05BD20A604A6C3E8D0E860A52D48A52C48A520852CA5E2
:2006200021852DA524A625205B06F003205B06A52C38E5B6A52DE5B7B042206D05F03DA6F5
:2006400028A52920A005A92020A604200C02B02C201404D0F32083064C2F0685B6E6B6D076
:2006600001E886B7A4C1C080F018206B04A52CA62D38E902B001CA852C4C480968852C6807
:20068000852D60A5BF30FBA90D200902AD1102297F85BFF007206409C6BFD0F9A90A4C61FA
:2006A00009AC120284BFB00BA930852C85C0842D20800545808580200602A000A6C0297FAE
:2006C000F0F1C97FF0EDC913F0DAC90AF0D3CD1002F009CD0F02D00AE030D016A62C84BF3D
:2006E000A90DE4C13008A90720A6044CB3069500E8E8CA86C0C90DD0BA208306209505852B
:20070000BC20950585BD6020D608206B0408206D0685B886B9A5BC85B6A5BD85B7A2002819
:20072000D00B206D05CACACA201404D0FA8428842920D608A90DD12CF011E8E8E8E8C8D1A8
:200740002CD0FAA5B68528A5B78529A5B885BCA5B985BD18A0008AF06E1029652E85B8A505
:200760002FE90085B9B12E91B8A62EE424D006A52FC525F04AE8862ED002E62FE6B8D0E57B
:20078000E6B9D0E1652485B8852E98652585B9852FA52EE5C6A52FE5C79005C62A4C140396
:2007A000B124912EA624D002C625C624A62ED002C62FCA862EE4BCD0E7A62FE4BDD0E1A5F8
:2007C000B88524A5B98525A5280529F017A52891BCC8A52991BCC884B620140408A4B69184
:2007E000BC28D0F24CCC02205403B5032980F002A9FF85BC85BD4875029502684875039531
:200800000368550185BB1003204308A011B5001501D0034C140338A5BCF50048A5BDF50179
:200820004845BD300A6885BD6885BC384C32086868183602360326BC26BD88D0D9A5BB1064
:200840000DA6C13898F500950098F501950160204108205403B50075029502B501750395E0
:200860000360205403A010B50285BCB50385BD1602360326BC26BD900D18B502750095026E
:20088000B5037501950388D0E660209505AAB500B401C6C1A6C194004C8705A27D20560334
:2008A000B50148B50048209505AA6895006895016020FD08A5BC852AA5BD852B60A22CD039
:2008C00002A22EB500C980B00DB501D009A52C852EA52D852F60A52CA42E842C852EA52DBA
:2008E000A42F842D852FA00060A52885BCA52985BD209C03A5C68526A5C7852760B1C68559
:20090000BC200809B1C685BDE6C6D002E6C7A522C5C6A523E5C7B0E44C140320240985BCBB
:20092000984C820520FC06A5BC85B620FC06A5BD85B7A4BC20FC06A6B7A5B6186CBC002034
:20094000420920F9044C8705862DE00060A00284BCA02984BDA000B1BCC908D0034C680310
:2009600060200902A9FF2C11023002A9004C0902243A912710E159C52A5610112C8B4C45C5
:20098000D4A080BD30BCE0131D9447CF8854CF30BCE0101116805355C230BCE01416905092
:2009A000D283494ED4E57188BBE11D8FA221586F83AC225583BA2493E0231D30BC20489128
:2009C00049C630BC313430BC84544845CE1C1D380D9A494E5055D4A010E7243F209127E1BD
:2009E0005981AC30BC131182AC4DE01D895245545552CEE0151D85454EC4E02D984C495385
:200A0000D4EC24000000000A801F2493231D30BCE15080AC59855255CE380A86434C4541D9
:200A2000D22B845245CD1DA080BD381485AD30D3176481AB30D385AB30D3185A85AD30D3D2
:200A400019542F30E285AA30E21A5A85AF30E21B542F98524EC40A8080120A09291A0A1ABD
:200A6000851813098012010B313061720B04020305031B1A190B09060A00001C172F8F5517
:200A800053D280A830BC312A312A80A92E2FA2122FC12F80A830BC80A92F83AC38BC0B2F45
:200AA00080A8522F84BD09022F8EBC84BD09932F84BE09052F09912F80BE84BD09062F8433
:0A0AC000BC09952F09042F00000067
:00000001FF
